:030000000219FDE5
:03000B000200AA46
:03002B000201656A
:03005B000202F8A6
:030073000202DEA8
:1000800002030406080C10182030406080040608A3
:100090000C10182030406080A0C000070F1F3F0DDB
:1000A0000D04050D050305030302C2AFC0D0C0E077
:1000B000206217E5256002E473E525F4F58A758B67
:1000C00000D262D0E0D0D0D2AF3285268AC262E5BB
:1000D00026F46035306803207210758B00D0E0D0B4
:1000E000D0C292C291C290D2AF32C292C291C2909B
:1000F000206E0C206609740AD5E0FDE57E429075FD
:100100008B00D0E0D0D0D2AF32758A00C28DD262DF
:1001100001FF01B9306805206602D29201B930684A
:1001200005206602D29101B9306805206602D2909E
:1001300001B9C29330680A2066077408D5E0FDD281
:100140009201B9C29430680A2066077408D5E0FDB0
:10015000D29101B9C29530680A2066077408D5E0CB
:10016000FDD29001B9C2AFC2AD53E6EFC0D0C0E03E
:10017000D2D3D2AFC2CEE52A6007207449152A2116
:10018000C67800790020742EE580307E01F430E4DA
:100190000278FF53DACF207E0343DA20307E034318
:1001A000DA10C2D8C271E580307E01F430E4027901
:1001B000FFC3E89970CB306103752A18207403756A
:1001C0002A18885FD27020740DE52B6004152B214E
:1001D000D643DA01C2D82070024134A85F20610200
:1001E000C2702074367982B70431C3E894F04003BA
:1001F00074F0F8E8C4540F28F87984B70302411B5F
:10020000C313C3138721200802C313200A06C3C8DF
:1002100098F8411B28F8500374FFF88822E52D5404
:10022000066011E533C313C31324062522F52250BB
:10023000037522FF7882B60459852224A824C3E5D9
:100240002495644002A864C3E895664002A86688C5
:1002500025E56970024185C3E8AA699A5003E8FA66
:10026000E4F9EAC333FBE56BF45B29400D256AF83A
:10027000E56A6002156A400B41850AC3E56A9A5037
:1002800002056A78FF8826C26EC3E52694F840020C
:10029000D26EC3E52594404002D26420CF0AD0E05C
:1002A000D0D043E610D2AD32C2CF053A7801E52A6C
:1002B0006005307402152AC3E55F9401400575623C
:1002C0000041D4756300756C00E5622401F562504D
:1002D000037562FFD0E0D0D043E610D2AD32C2AF9A
:1002E000C0D053E67FC260759100855694855795BE
:1002F000759104D0D0D2AF32C2AF53E6EFC2ADC0D9
:10030000D0C0E0C0F0D2D3D2AFA8FBA9FCC2D83095
:100310007102615F53DACF207E0343DA10307E032F
:1003200043DA20D271E580307E01F420E4026136A8
:1003300088278928A18C53DACF207E0343DA203026
:100340007E0343DA10C2D8C271307402A1787800FB
:10035000E580307E01F430E402A178885FA160532B
:10036000DACF207E0343DA20307E0343DA10C271F5
:10037000206102813853DACF207E0343DA10307EC9
:100380000343DA20C2D8D271885A895BC3E89558F2
:10039000F8E99559F97B007E087A00C3E8948CE966
:1003A00094005005755E00812A882178A2E6A82174
:1003B0006055C3E894C8E994005008E4D2E4FB7A9D
:1003C0000A8105C3E89468E994015008E4D2E3FB8C
:1003D0007A0F8105C3E894D0E994025008E4D2E290
:1003E000FB7A1E8105C3E894A0E994055008E4D285
:1003F000E1FB7A3C8105C3E89498E994085008E44D
:10040000D2E0FB7A787E00C3E8955CFCE9955DFD5F
:1004100030E70AECF42401FCEDF43400FD755E00D5
:10042000C3EC9AED9E5003755E01885C895D855A28
:1004300058855B597802A160C3E89527F8E99528AB
:10044000F9307C02A144307B02A144307A02A13D04
:10045000207502815BE9FDE8FC817AE9C313F9E8C4
:1004600013F8307902A13DE9C313F9E813F83078A5
:0F04700002A13DE9C313FDE813FC20612CC3EC8E
:10047F00941CED940240028191ED701EC3EC94C860
:10048F0050180529E52970021529C3E529940A504A
:10049F0002A178755F00D270A178E5296002152955
:1004AF007888E6F97400207F087896B90302789E61
:1004BF00E624FAFEE43400FFC3EC9EFCED9FFD92B0
:1004CF0008B90310A2085007207609D27681E330CD
:1004DF007602C276A2085016B9030DECF42401FC83
:1004EF00EDF43400FD0204FD78007900A144B90356
:1004FF0015EC33FCED33FDC3EC940AFCED9400FDD9
:10050F0050047C007D00C3EC94FFED94004006780E
:10051F00FF7900A144EC8575F0A4C5F0A2F733F87C
:10052F007900400302056078FF7900020560E9C396
:10053F0013F9E813F8307C0EE9600278FFC3E81373
:10054F0038F8E43400F9C3E894FFE99400400278E6
:10055F00FF885FD270206102A178741FF4552F4B72
:10056F00F52FC274EB7002D274752A1830740375AC
:10057F002A0A306102A18C20740353DAFE2074031F
:10058F00752B06D0F0D0E0D0D0D2AD43E610327943
:10059F00010205BC79030205BC790A0205BC791E6C
:1005AF000205BC79640205BC79C80205BC7817E462
:1005BF00D5E0FDD8FAD9F6227A147B780205E37AD2
:1005CF00107B8C0205E37A0D7BB40205E37A0B7B7B
:1005DF00C80205E37902B27DE4C294D5E0FDD29161
:1005EF00D5E0FDC291D5E0FDD294D5E0FDD292E5E4
:1005FF0076D5E0FDC2927496D5E0FDD9D9EAF8D54B
:10060F00E0FDD8FBDBCEC29422C37C007D0075F0E9
:10061F000005F0EA33FAEB33FB50F6EB13FBEA136A
:10062F00FAC3E9FFE8FEE89AF8E99BF95004EFF9FD
:10063F00EEF8B3EC33FCED33FDD5F0DFEDF9ECF86C
:10064F0022E889F08A20D2D4F8A9F07B0030F70B8A
:10065F007BFFF42401F8E9F43400F9E88520F0A4D5
:10066F00ADF0F8E98520F0A4AFF0FEED2EF974009F
:10067F003FFA7C04C3EA13FAE913F9E813F8DCF440
:10068F008BF030F70AE8F42401F8E9F43400F9E8C4
:10069F0089F0C2D4F8A9F0227882B60403020702C7
:1006AF00C3E55F940140030206CC852224E4F5459F
:1006BF00F546F547F548F549C26D0207027882E61F
:1006CF00FCD26DE522F523783879C7AA40AB41C338
:1006DF00EB13FBEA13FAEC146013C3EB13FBEA13EF
:1006EF00FAEC14146007C3EB13FBEA13FAD1188862
:1006FF0045894622C3E5459523F8E5469400F95010
:10070F000CC3E89480E994FF4016020733C3E894C2
:10071F007FE994005003020733787F790002073393
:10072F00788079FF884A894B22E54A2547F8E54BBF
:10073F003548F9854B20E4300701F43549FA30E7A5
:10074F0009C3EA94F04015020771C3EA940F5003EE
:10075F0002077178FF79FF7A0F020771780079002D
:10076F007AF0C3E5249564500AC374019524500BA5
:10077F0002078FE54B20E70E02078FE54B30E706A8
:10078F00884789488A492278A4E6FAC3E54A33F8AC
:10079F00E54B33F9D150E930E70BC3E89480E99486
:1007AF00FF4013E1C9C3E8947FE994005002E1C907
:1007BF00787F7900E1C9788079FFE820E715C3E5F4
:1007CF002398F84009C3E8940140030207F0780129
:1007DF000207F0E8F424012523F840030207F0781C
:1007EF00FF884C2278A5E6FAA848A949D150E930EC
:1007FF00E70CC3E89401E994FF4016020824C3E80C
:10080F0094FFE99400500302082478FF790002084E
:10081F0024780179FFE920E715C3E54C98F84009E2
:10082F00C3E89401400302084B780102084BE8F437
:10083F002401254CF8400302084B78FF88242278C6
:10084F00FFC26420693D206A12D264C3E541940A55
:10085F004009C3E52594405002C26479A1E76023A3
:0D086F00E541601F74FF8541F0848539F07C
:10087C00306A0375F005A4F8C5F0600278FFC3E890
:10088C0095675002A867886622C3E5409440E5410D
:10089C009401E56650031401A6046002F566220279
:1008AC0008AE2275E890227883E6FFE5E820ECF7A5
:1008BC00A8BDA9BE0573C3E57394084052757300B7
:1008CC00E9FA79A0E76044EA7007E574601B020856
:1008DC00E9C3E895746010E5745006600C140208C6
:1008EC00F50460F90208F5E574F574C39458401BDF
:1008FC007564C0C394044013756480C39404400BA6
:10090C00756440C39404400375640075BB0322E511
:10091C00642410500274FFF5647982B704022142FA
:10092C00C3A864E524985002A824C3E89566400245
:10093C00A86688258826E573B4070375BB10227456
:10094C003279A687F0A4C5F0A2F733F8C3E8956412
:10095C004002A86488228824882588268867227506
:10096C0040007541F022C2AF75C820A8CCA9CDAA11
:10097C003A30CF010A75C824D2AFAB3BAC3C883BB4
:10098C00893CC3E89BF8E99C206908F9306702416F
:10099C008721E4AD3D8A3DF9EA9DFA600478FF7940
:1009AC00FFAE3EAF3F8B3E8C3FC3EC9FFCC3E99C3C
:1009BC00F542A83BA93CC3E89EF8E99FF9C3E54181
:1009CC0013FBE54013FAE82AF540E93BF5415006E4
:1009DC007540FF7541FF412EAA40AB41AC40AD4183
:1009EC007E047F02C3EB940440021E1FC3EB9408E9
:1009FC0040021E1FC3ED13FDEC13FCDEF7C3EA9C93
:100A0C00FAEB9DFBEF6009C3E913F9E813F8DFF784
:100A1C00EA28FAEB39FB8A408B4150067BFF8B406E
:100A2C008B41C3EB94025002D2673069047F0341BF
:100A3C00597892E6FFC3E537948240110FC3E5372E
:100A4C0094A040010FC3EF940640027F057E05E59C
:100A5C0041C4540FF9E541C454F0F8E540C4540FB7
:100A6C0028F8C3E89EFAE99400FB4009C3EA940213
:100A7C00EB940050047A02E4FB41D3AA40AB41EB67
:100A8C00C4FEEAC4540F4EFCC3EA9CFAEB9400FB80
:100A9C00C3E813C313F8EA28FAEB3400FB8A408B43
:100AAC0041C3EB94024002C2677805EBC4FE7B00A5
:100ABC00EAC4540F4EFAC3EA98FA4005C3940250A4
:100ACC00027A027892E6FF30600241D38552568555
:100ADC005357D26043E680C3E49AF8E49BF930673D
:100AEC0002616DE8FAE9FBD3E913FDE813FC8852C7
:100AFC008953C3EF94036038EF20E00DE82CF8E93C
:100B0C003DF9ECFAEDFB020B28E828F8E939F9C3BA
:100B1C00E82402F8E93400F97AFE7BFFC3EF940372
:100B2C00400E8A548B55884E894F8C508D5161A143
:100B3C00885489558A4E8B4F8C508D51306920C307
:100B4C00E53394034019E542A2E713F8E555F42484
:100B5C000138400B20E7087554FFF42401F555616A
:100B6C00A1E8FAD3E813FC8852C3EF94036020EF9A
:100B7C0020E007E82CF8ECFA618DE8282402F87ADA
:100B8C00FEC3EF940340088A54884E8C5061A188B0
:100B9C00548A4E8C50E56BC3335002646BF56B304A
:100BAC00600261AB753402D26043E680E52D5406D9
:100BBC006026A840A941C3E913F9E813F8C2AF5362
:100BCC00E67F759100C3E498F594E499F5957591D9
:100BDC0004D26043E680D2AF22D265754400752002
:100BEC0000306B03752040020C04D265754400750F
:100BFC002040306B03752000D2AF7801206722E5CE
:100C0C002D54066002C265C3E54194054013780279
:100C1C009405400878039405400278063069027800
:100C2C000A206019E544601530690AC3E533940362
:100C3C004003D53406D2AFD26C81D671B3D2AF009B
:100C4C0000C2AF206726E541C3FB940F40027B0F27
:100C5C00EB240530730123306A02742820620123CF
:0E0C6C00F93069027982E58BC39940B50544E1
:100C7A00E59BF45440B5200281C030690A08C3E8F4
:100C8A00940A400108812D2065028104C26553E659
:100C9A007F7591003067107594007595FE75910403
:100CAA00D26043E6808104AE40AF41C3E49EF5942E
:100CBA00E49FF59581A7C3E533940250028104307D
:100CCA0065028104D80281D4812DC26C53E67F75F6
:100CDA009100855494855595759104854E56854F96
:100CEA0057D26043E680D2AFE52D54066008206AE9
:100CFA00020533020D10306C0D206B0A20650715B2
:100D0A0081158102157B22780030640530650278EE
:100D1A0001E53775F007A4F9E5F028F5F0E9A2F046
:100D2A0013A2F113A2F213F537C39478500375375F
:100D3A0078C3E53795384008D266C292C291C2900C
:100D4A00306002A14A855056855157D26043E680E9
:100D5A0022207D11C2AF754302C294D293D2AF75DD
:100D6A009F10020F2AC2AF754302C294D295D2AF26
:100D7A00759F10020F2A307243207D20C2AF75433F
:100D8A0003900143757E10C290C295306204D291DD
:100D9A00A19ED294D2AF759F20020F2AC2AF75438B
:100DAA0003900143757E10C292C293306204D291BD
:100DBA00A1BED294D2AF759F00020F2A207D17C21E
:100DCA00AF75430390011EC290306202D291D2AF36
:100DDA00759F20020F2AC2AF75430390011EC2926B
:100DEA00306202D291D2AF759F00020F2A207D1184
:100DFA00C2AF754304C293D295D2AF759F00020F5A
:100E0A002AC2AF754304C295D293D2AF759F20020E
:100E1A000F2A307243207D20C2AF754305900132FC
:100E2A00757E08C291C294306204D292C13AD293BA
:100E3A00D2AF759F10020F2AC2AF754305900154B5
:100E4A00757E20C291C294306204D290C15AD29562
:100E5A00D2AF759F10020F2A207D17C2AF754305C6
:100E6A00900114C291306202D292D2AF759F1002E1
:100E7A000F2AC2AF754305900128C2913062EBD2A6
:100E8A0090D2AF759F10020F2A207D11C2AF754311
:100E9A0006C295D294D2AF759F20020F2AC2AF75AF
:100EAA004306C293D294D2AF759F00020F2A3072C2
:100EBA0042207D20C2AF754301900154757E20C245
:100ECA0092C293306204D290C1D6D295D2AF759FA6
:100EDA0000020F2AC2AF754301900132757E08C223
:100EEA0090C295306204D292C1F6D293D2AF759F66
:100EFA0020E12A207D16C2AF754301900128C292D3
:100F0A00306202D290D2AF759F00E12AC2AF754318
:100F1A0001900114C290306202D292D2AF759F2022
:100F2A00C26622900112757E00C292C291C290C21C
:100F3A0093C294C295C2622278807609087609081B
:100F4A0076040876FF0876030876FF08760B08769B
:100F5A0003087601087601788C76010876FF087610
:100F6A00FF0876FF0876FF0876FF0876030876FF03
:100F7A000876FF0876FF0876250876D008762808CE
:100F8A0076500876040876FF087602087600087616
:100F9A007A0876FF08760108760108760008760353
:100FAA00227887E6FFC272BF0302D2727888E6C34C
:100FBA0094036008C27DE630E102D27DC27E788960
:100FCA00E630E102D27EC3EF94026008758E01D248
:100FDA0073020FE3758E00C273227880E6149000C4
:100FEA00809378A4F67881E6149000809378A5F629
:100FFA007886E61490008D9378A6F6789CE6753884
:10100A00FF75390CB402067538A075390AB403069F
:10101A0075388275390578A3E61490009A93F569B4
:10102A00120F2D22227896E6FA7897E6FB7888E660
:10103A00B40305C3EB940EFB307F047A007BFFC335
:10104A00EB9AFCC3948250027C827575000575EC9C
:10105A008575F0A4C3E5F0947D40F222D27F112F6A
:0F106A001205AD7A007B007C101205A3E55F2A0A
:10107900FA74003BFBDCF37C04C3EB13FBEA13FAC1
:10108900DCF7FEC27F112F22E5EF20E60375200071
:101099000520903FFFE520146006901DFF146000B5
:1010A9009304600375EF1253D9BF7581C043FF8064
:1010B90012059E75EF0243B203E5B3240420E70D40
:1010C900F521E5E320E0068521B343E301120F2D65
:1010D9007580FF75A40075F1D475D4EF7590C0754E
:1010E900A53F75F2FF75D50075A60175E241E4F8D3
:1010F900F6D8FD756B01120F421215BD78988676E8
:10110900753001C2AF1205B71205C71205AD120538
:10111900CE1205AD1205D51205ADC2AF78FA79FA2E
:10112900308407D9FBD8F7021C00120FAB120FE469
:10113900112E112F78988676120F2D758850758982
:101149001275C82475910475D84075A82275B8021E
:1011590075E690759B80759D0075D10E75BC5875A7
:10116900BB0375BA1175E88012059ED2AF1208ABA0
:1011790053DACF207E0343DA20307E0343DA10436B
:10118900DA01C2D8C2711205B7D2617B037A0CE5C4
:101199005E70077A0CDB030211231205AD20700380
:1011A900021123C270E55FC3940240E1E52F541F89
:1011B900856160F561B560D5DAD5C26153DACF20B2
:1011C9007E0343DA20307E0343DA10C2D8C2717835
:1011D900A2E67008D274E52F54E0F52FC27575297F
:1011E900001205B2307409C3E529940A4002D27588
:1011F9001205A378023074027800C3E55F9840F0C5
:10120900C2AF1205C71205C71205C7D2AF1205B77B
:10121900754D007888E6B4030241FA1205A3788C6B
:10122900E6C3940150030212FAE530C39401500356
:101239000212FA207435C3E55F94FF50030212FAD3
:10124900C2AF1205DCD2AF1205B2C3E55F940150FB
:10125900EFC2AF1205C71205A81205C7D2AF120512
:10126900B2C3E55F94FF40E90217657F02D27F119F
:101279002F1205B2C2AFC27F112FAE5FC3E55F94D3
:101289007FD2AF407612059EC2AF1205DCD2AFDF26
:10129900DC1166C3EE94057897F61205B71215FFAF
:1012A9001216E87F0AD27F112F1205B2C2AFC27F90
:1012B900112FAE5FC3E55F947FD2AF50E612059E52
:1012C900C2AF1205C71205A81205C7D2AFDFD611E2
:1012D90066EE24057896F61205B71215FF12171750
:1012E9001205B2112FC3E55F94FF5002413C02176A
:1012F90065C3E55F954D4003855F4D1205B27801E1
:101309007988E7B403027805C3E55F984002411C78
:10131900C2AF1205DC1205DC1205DCD2AF1205B72B
:10132900753000E4F531F5320531E531F4703905F0
:1013390032789AE67819146012783214600D787D43
:1013490014600878FA146003753200C3E5329840D6
:101359001715327531B478998676C2AF1205DCD289
:10136900AF789886761205B21205A8E52A7005307D
:101379007402212378012074027806C3E55F98403E
:10138900A77888E6C3940360031205B2E52A7003BF
:10139900021123C2AF120F2DE4F522F523F524F52E
:1013A90025F526F56AD2AF7885E6C333F568E4F505
:1013B90045F546F547F548F549F573F52CF52DF54D
:1013C9003775730875BB1012059E1208AFE5E82042
:1013D900ECFBA8BDA9BEE97001F888741208B375C1
:1013E900730875BB107887E6FE7602120FAB788713
:1013F900EEF6C2AF7564FF12094B8522648522653A
:10140900852266D2AF7522017524017525017526DD
:101419000185636C756D017888E6B40307C27D3078
:101429007602D27DD268D269753300120E93120EFC
:10143900B812096B12097212096B12097212096B3F
:10144900021459C2AF120FABD2AF75730075BB034B
:10145900120BF61206A7120D11120D5B1209721268
:0E1469000BE5306D0312070320670312084ED7
:10147700306703120895120D11120D8012097212AE
:101487000BF6306D03120738120D11120DF7120902
:1014970072120BE5306D03120796120D11120E1C16
:1014A700120972120BF6306D031207F3120D1112A7
:1014B7000E931209721208AF120BE5120D11120EDC
:1014C700B81208B3120972306935206B3285676428
:1014D70085676585636C756D0179187A0CC3E5338B
:1014E70099400FC269D26A8A358567648567660243
:1014F7001506C3E55F9401400302145902158330B2
:101507006A1B206B18E535147004C26A814CF535E7
:10151700C3E55F9401400302145902158375360031
:10152700C3E56278FA985054307404E52A604D7820
:1015370088E6B40317207D05207607A1533076028D
:10154700A153206B07D26B856764819878F0306B65
:10155700058567647820C3E5419850028159306B4F
:101567001BC26BC27D307602D27DD26A7535128579
:10157700676481590536E55F6002A186753600C24A
:10158700AF120F2D7887E6FE7602120FAB7887EE43
:10159700F6E4F522F523F524F525F526F568C26866
:1015A700D2AF12059E120F2D307409C3E53694058C
:1015B70040022123612C901A0D7820121641E52054
:1015C700B4550CA3121641E520B4AA030215DF1285
:1015D7000F421215FF0215FE901A0378807B0A123C
:1015E7001641A308DBF9901A0F788C7B1812164165
:1015F700A308DBF9901A2722C2AF12168012165AD7
:10160700901A00740E121646A37404121646A37499
:1016170014121646901A0378807B0A121645A308FF
:10162700DBF9901A0F788C7B18121645A308DBF9A3
:10163700121693121671901A2722E493F622E643A4
:101647008F01538FFD75EF0275B7A575B7F1F0538D
:101657008FFE22438F02438F0175EF0275B7A57581
:10166700B7F1901A0DF0538FFC22901A0D7455D1D3
:1016770046901A0E74AAD146227A3079D0782090F3
:101687001A40D141E520F709A3DAF7227A3079D059
:10169700901A40E7D14609A3DAF922AB77A878BBBD
:1016A70001027980BB02027981BB03027982BB0404
:1016B700027984BB05027986BB06027992BB0702D1
:1016C7007987BB080279A3BB0902799CBB0A027917
:1016D70088BB0B027989E8F7227C051205B7DCFB8A
:1016E70022C2AF1205C71205CE1205D51205DC12AC
:1016F70005A81205C71205CE1205D51205DC12057D
:10170700A81205C71205CE1205D51205DCD2AF22E5
:10171700C2AF1205DC1205D51205CE1205C7120598
:10172700A81205DC1205D51205CE1205C71205A8A9
:101737001205DC1205D51205CE1205C7D2AF22AEAF
:1017470077AF78C2AF1205C71205C71205C71205D2
:10175700A8DEF21205DC1205A8DFF8D2AF22D1E825
:10176700D1E0D1E0757701757801757900F1467C94
:1017770005AD5F1205B7C3ED955F70F5C3E55F94DF
:1017870001400AC3E55F94FF40320217A1D1A2B11D
:10179700FFD1E8C2AF75EF12D1E0DCD50579C3E51B
:1017A700799403500280C6D1E00578E5771490005C
:1017B7009F93F808C3E57898500280AED1E0D1E056
:1017C7000577C3E577940C5002809C120F42B1FF56
:0717D700C2AF75EF12D1E073
:0319FD0002109144
:101A00000E0414090904FF03FF0B03010155AA0189
:101A1000FFFFFFFFFF03FFFFFF25D0285004FF0259
:081A2000007AFF01010003FF41
:101A400023484B696E67313041232020202020201D
:101A500023424C48454C4923463333302320202031
:101A60002020202020202020202020202020202076
:101C0000C2AFC2D353D9BF7581C043B20343FF8073
:101C1000752438752503B1C975EF0275E24043F1AB
:101C20001053A4EF75D400D2847DFA780379E67C52
:101C300010752200752300901DD67B0675249875BB
:101C400025013084028142208408D8FBD9F9DCF7D1
:101C500081B4308408D8FBD9F9DCF781B4B189E4C8
:101C600093A3C39A6004DDC381B4DBDBB17B600264
:101C7000812B7B08E493FAA3B15CDBF87A30B15C8A
:101C8000752200752300B17BEAFCEBFDC3ED94FEE9
:101C9000400EB17B8A278B28ED30E0048A828B834B
:101CA000B17B7AC270D8C3ED94FE601350CEBD00F4
:101CB00025EC60097520007521FF0200008100A855
:101CC00027A9280809D804D90281D3B17FEA89AAB3
:101CD000F281C50D81A0C3ED94035049EDA2E092BD
:101CE000007AC5C3E5829400E583941C50902000DF
:101CF00010438F02438F0175B7A575B7F1F030001F
:101D00001FA827A9280809438F01538FFDD804D99C
:101D100002A12089AAE275B7A575B7F1F0A3A10DBC
:101D2000538FFC817C7AC1BD030CE493A3FAB140CC
:101D3000DCF8B138817C817EAA22AB23B15CEBFA5E
:101D4000EA6222752608C3E52313F523E52213F57D
:101D50002250066323A0632201D526EAB1C9B1C986
:101D600075260AEAF4200102D284300102C284B14D
:101D7000C9C3134002C201D526EB22B17FEAFB2082
:101D80008402A17F308402A184752608AE24AF2589
:101D9000C3EF13FFEE13FEB1CDB1C9C3EA13308414
:101DA000024480FA30E703632201C3E52313F523DD
:101DB000E52213F52250066323A0632201D526D91C
:101DC000E52265236523F52222AE24AF250E0FDE22
:101DD000FEDFFCD20122424C48656C693437316326
:041DE000F3300601D5
:00000001FF
